:1000000012C02CC02BC02AC029C028C027C026C0BF
:1000100025C024C023C022C021C020C01FC01EC0D4
:100020001DC01CC01BC011241FBECFE5D4E0DEBF25
:10003000CDBF10E0A0E6B0E0E8E9FBE102C005902A
:100040000D92AA37B107D9F710E0AAE7B0E001C0D6
:100050001D92AE3CB107E1F7CCD79CCDD1CF8064E7
:1000600087B920E030E040E0369A3699FECF84B17F
:1000700095B1280F391F4F5F4431B1F7C90164E1D1
:1000800070E052DDCB010895482F440F662359F0EC
:1000900028B381E090E0042E02C0880F991F0A94D3
:1000A000E2F7282B28BB87B321E030E002C0220F03
:1000B000331F4A95E2F7822B87BB84EC99E00197C6
:1000C000F1F787B32095822387BB662319F088B3A5
:1000D000282328BB08958F929F92AF92BF92CF9210
:1000E000DF92EF92FF920F931F93CF93DF93D82E5F
:1000F000C62E80917F00D81629F48091AE00681733
:1001000009F486C1AD2CBB24C501880F991F42E0BC
:1001100050E0082E02C0440F551F0A94E2F74093A6
:100120008E0021E030E0B90102C0660F771F8A958A
:10013000E2F7862E6093800015BA18BA17BA0C2C15
:1001400002C0220F331F0A94E2F7922E24BB47BB52
:1001500002EE14E0C8010197F1F78D2D80DF909336
:100160009B0080939A008D2D61E08EDF8D2D77DFCF
:1001700090939F0080939E00C8010197F1F78D2D09
:100180006EDF90939D0080939C00A89520919A002B
:1001900030919B002F5F3F4F2817390740F0809127
:1001A0009E0090919F002817390708F028C1809180
:1001B000800087BBC0E0D0E0FF2407C0A89521964F
:1001C00021F4F3947EE1F71649F08D2D48DF8C0180
:1001D0008C2D45DF0A968017910780F3809180006F
:1001E00088BB82EE94E00197F1F78D2D38DF909374
:1001F0009F0080939E0080E29EE40197F1F78D2D91
:100200002EDF9C019093A1008093A00080919E001E
:1002100090919F0003962817390728F483E0223530
:10022000380708F4F5C080917C00882321F0275B13
:10023000334008F0EDC018BAC0E0D0E0FF2407C09A
:10024000A895219621F4F3947EE1F71649F08D2DBF
:1002500006DF8C018C2D03DF0A968017910780F34F
:1002600087E084BB8091800088BB81E090E002C081
:10027000880F991FAA94E2F7982F80938000E4EFEB
:10028000F1E03197F1F794BA20E030E060E008C087
:10029000A8952F5F3F4F21F46F5F6E3109F43CC08A
:1002A00083B38923A9F3E62E6623B1F52F3F3105E9
:1002B00009F090F518BAFF24C0E0D0E007C0A89577
:1002C000219621F4F3948EE1F81649F08D2DC7DEC6
:1002D0008C018C2DC4DE0A968017910780F387E08D
:1002E00084BB15BA80918E0087BB88BB84EF91E0F8
:1002F0000197F1F794BA9091800020E030E008C0B7
:10030000A8952F5F3F4F21F4E3946EE1E616D9F0F4
:1003100083B38923A9F378C088EE93E0A0E0B0E02E
:100320008093810090938200A0938300B093840017
:100330007BE1E72E71E0F72E012D112D17C025303E
:10034000310508F45CC081E090E0A0E0B0E080936B
:10035000810090938200A0938300B09384006E2D5F
:100360005AE8E52E51E0F52E012D112D70E080E0C8
:1003700090E0CB017727662740E050E0620F731FC3
:10038000841F951FA8019701B0DB24E630E040E010
:1003900050E0DEDB609181007091820080918300EB
:1003A00090918400A2DB609381007093820080931F
:1003B00083009093840087E080937E00D092AE000B
:1003C000C0927F0087BA18BAC0E0D0E0FF2407C00F
:1003D000A895219621F4F3947EE1F71649F08D2D2E
:1003E0003EDE8C018C2D3BDE0A968017910780F350
:1003F00087E084BB85BB84EC99E00197F1F714BAE0
:1004000015BA17BA18BA04C0EE2009F498CF9BCFDA
:10041000DF91CF911F910F91FF90EF90DF90CF90E0
:10042000BF90AF909F908F9008952F923F924F92E0
:100430005F926F927F928F929F92AF92BF92CF9274
:10044000DF92EF92FF920F931F93DF93CF93CDB77D
:10045000DEB727970FB6F894DEBF0FBECDBF782E5C
:10046000662E942EA895262F30E03F832E83220FF0
:10047000331F3D832C8391E0492E512CC2010C8007
:1004800002C0880F991F0A94E2F7182F87BB18BA89
:10049000472D50E05B834A83C2010A8002C0880F67
:1004A000991F0A94E2F7898384BB85BB82EE94E0AE
:1004B0000197F1F7892D60E0E7DD862DD0DD4497C7
:1004C00040F0892D61E0E0DD862DC9DD449708F01C
:1004D00039C1E92CEE0C27B381E0A82EB12CC5015F
:1004E0000E2C02C0880F991F0A94E2F7C82E282B01
:1004F00027BB84EF91E00197F1F7862DB0DD8D5B8E
:10050000924008F449C017BB87B3E3940E2C02C095
:10051000AA0CBB1C0A94E2F7EA948A2987BB84ECF4
:1005200099E00197F1F7862D9ADD5C01892D97DD21
:10053000AC0117BB20917E00822F8250823018F4CC
:1005400081E080937B00E0917B00F0E0EE0FFF1FE5
:10055000DF01A155BF4FAD92BC92EE55FF4F5183C5
:100560004083493C510530F0253061F082E08093B2
:100570007E0006C0253031F083E080937E0082E06B
:1005800080937D0080917E00853031F090927A00DA
:10059000609299007092B30015BA8A81880F21E0A9
:1005A00030E0190102C0220C331C8A95E2F78C2D31
:1005B000822987BB88BB29010E8002C0440C551CD0
:1005C0000A94E2F744BA04EC19E0C8010197F1F784
:1005D000872D45DD845F914008F0B1C080917B009C
:1005E000813009F42EC3822C28BAC8010197F1F793
:1005F00027BA12EEA12E14E0B12EC5010197F1F732
:10060000872D2DDD8C0118BAC5010197F1F728BAA5
:10061000C5010197F1F7872D22DD045F114008F035
:1006200046C08558934008F442C085E080937E0020
:1006300017BA18BA45BAC5010197F1F727BAC5012B
:100640000197F1F7872D0BDDC39708F072C087B3D0
:10065000C82AC7BAC5010197F1F7892D00DD883C8A
:10066000910508F466C0872DFADC8639910508F4F7
:1006700060C027BAC5010197F1F7872DF0DC8639F4
:10068000910508F456C028BAC5010197F1F718BAC8
:10069000C5010197F1F7872DE2DCC39708F049C047
:1006A00084E080937E0081E080937B0042C027B38A
:1006B000E39481E090E002C0880F991FEA94E2F78A
:1006C000282B27BB28B3822B88BB84ED90E30197AE
:1006D000F1F7872DC4DC8C01892DC1DCAC0188BA0F
:1006E00087BA80917E008250823018F481E0809336
:1006F0007B00E0917B00F0E0EE0FFF1FDF01A155D2
:10070000BF4F8FEF93E09C01201B310B2D933C9347
:10071000EE55FF4F841B950B91838083445F5140BE
:1007200010F482E001C083E080937E0081E080933A
:100730007D0090927A00709299006092B30014BA92
:1007400015BA6AC187B3992D990F02E010E002C073
:10075000000F111F9A95E2F7802B87BBA8E8AA2EFD
:10076000A3E1BA2EC5010197F1F7862D78DC7C0153
:1007700088B3082B08BBC5010197F1F7862D6FDC04
:1007800024E630E0E20EF31EE816F90690F515BAFD
:10079000C2010E8002C0880F991F0A94E2F784BB41
:1007A00097B38A81880F02C0440C551C8A95E2F7E2
:1007B000842D942997BB98B3892B88BBC5010197D9
:1007C000F1F7892D4CDC8152934020F083E0809337
:1007D0007E0004C083E080937E0085E080937D00EE
:1007E00081E080937B0090927A00709299006092F1
:1007F000B30015BA01E010E0C8010E8002C0880FF6
:10080000991F0A94E2F7C82E84BBAA80BB80AA0C69
:10081000BB1C87B30A2C02C0000F111F0A94E2F719
:10082000902F802B87BB88B3982B98BBE8E84E2E7F
:10083000E3E15E2EC2010197F1F7872D10DC7C0108
:1008400008BBC2010197F1F7872D09DC8C599F4F36
:100850008E159F05F8F4498145BB44BBC201019741
:10086000F1F7892DFCDB883C910528F483E0809327
:100870007E0084E004C083E080937E0086E0809365
:100880007D0081E080937B0090927A0060929900D5
:100890007092B30002E010E00A2C02C0000F111F9A
:1008A0000A94E2F771E0E72EF12C02C0EE0CFF1C77
:1008B000AA94E2F715BAC4BA892D61E0E5DB62EECD
:1008C000C62E64E0D62EC6010197F1F7872DC7DB4F
:1008D0005C01862DC4DBA81AB90A07BB08BBC60198
:1008E0000197F1F7872DBBDB1C01862DB8DB2C01AE
:1008F000E7BAE8BA892D60E0C7DBC6010197F1F7D6
:10090000872DADDB4C01862DAADB881A990A07BB1F
:1009100008BBC6010197F1F7872DA1DB8C01862D5D
:100920009EDB8A149B0420F481010419150903C07D
:10093000081B190B5401C5014F978759934008F0C4
:100940006BC080917E00882311F0863019F481E01D
:1009500080937E0020917C00E22FF0E0EE0FFF1FDD
:10096000EE0FFF1FEC54FF4F7082618286E390E030
:10097000DC01AA9EC001AB9E900DBA9E900D112481
:100980006BE070E0D1D8738362832F5F20937C008B
:1009900046E0000F111F4A95E1F7C50165E070E0E0
:1009A000C3D85B0160E034C0E62FF0E0EE0FFF1F1C
:1009B000EE0FFF1FEC54FF4F8081861541F58181BA
:1009C000871529F50A151B0510F5362F422F50E023
:1009D0004150504016C0EE0FFF1FEE0FFF1FDF010A
:1009E000AC54BF4FE854FF4F80818C9381811196A6
:1009F0008C9311978281938113969C938E93129777
:100A00003F5FE32FF0E0E417F5072CF322506F5F10
:100A1000621750F220937C002A813B81220F331F02
:100A200062E0E62EF12C6701022E02C0CC0CDD1C28
:100A30000A94E2F701E010E0F80102C0EE0FFF1F98
:100A40002A95E2F715BAC8010E8002C0880F991FD7
:100A50000A94E2F784BBE7BBE8BB862D00DB5C01B0
:100A6000872DFDDA4C018A189B08C7BAC8BA862DB3
:100A7000F6DA6C01872DF3DA2C014C185D080C8036
:100A800002C0EE0CFF1C0A94E2F70C8002C0000FBB
:100A9000111F0A94E2F7F981F4BBF5BB18BA07BB42
:100AA000872DDDDA2FEF33E0A20EB31EA81AB90AA4
:100AB000E7BA872DD4DA860101501C4F081B190BA9
:100AC000C4018A199B098458934030F4C201801BE9
:100AD000910B459708F0B5C0C20155E0880F991FEA
:100AE0005A95E1F76FE170E01FD86815790508F0B5
:100AF000A8C080917E00823018F0863009F0A1C035
:100B0000A091CC00A63009F07EC08091CD00861562
:100B100009F079C080918500871509F074C0609153
:100B2000AA007091AB00EBE0F0E08E9EC0018F9EBA
:100B3000900D9E9E900D1124845B9B4F9B01220F74
:100B4000331FAB01B3E0440F551FBA95E1F7240FF3
:100B5000351F28513C4F8217930708F44FC06E9FF2
:100B6000C0016F9F900D7E9F900D1124845B9B4F61
:100B70009401220F331FA40163E0440F551F6A95AF
:100B8000E1F7240F351F28513C4F82179307B0F12E
:100B90006091AC007091AD004E9EC0014F9E900DD3
:100BA0005E9E900D1124845B9B4F9B01220F331F8F
:100BB000AB01B3E0440F551FBA95E1F7240F351F81
:100BC00028513C4F82179307C8F06E9FC0016F9F5A
:100BD000900D7E9F900D1124845B9B4F9201220FFC
:100BE000331FA201F3E0440F551FFA95E1F7240FDC
:100BF000351F28513C4F8217930718F41092CC00F0
:100C000020C0A0937E009092AB008092AA005092E8
:100C1000AD004092AC008FEF93E09C012A193B0994
:100C20003093960020939500801B910B9093980031
:100C3000809397007092CD006092850086E080934B
:100C4000CC0014BA15BA17BA18BA27960FB6F8948A
:100C5000DEBF0FBECDBFCF91DF911F910F91FF90EF
:100C6000EF90DF90CF90BF90AF909F908F907F904C
:100C70006F905F904F903F902F900895EF92FF926A
:100C80001F93CF93DF93EC01162F633088F461300C
:100C900039F480E690E0A6D680E357D6888106C076
:100CA00080E690E09FD6888150D689814ED61CC0C0
:100CB00010927B00E42EFF2413C090E002968E1564
:100CC0009F0511F48EE241D680917B00FE01E80F72
:100CD000F11D80813AD680917B008F5F80937B00ED
:100CE00080917B00811748F3DF91CF911F91FF9096
:100CF000EF900895DF92EF92FF920F931F93CF939F
:100D0000DF9380919900E82FF0E09F01220F331FBD
:100D1000A1E0B0E0CD0102C0880F991F2A95E2F74B
:100D20009C0110917A00612F70E0AB01440F551FB8
:100D300082E090E002C0880F991F4A95E2F7982F51
:100D4000922B90938000322F20938E0097BBAD01A1
:100D50000090B30002C0440F551F0A94E2F7ED0162
:100D6000012E02C0CC0FDD1F0A94E2F7BE01642BF6
:100D700064BB80917E00833009F0DFC080917D00EC
:100D8000813009F067C015BA98BBCD0102C0880F49
:100D9000991FEA95E2F7982F80938000E4ECF9E040
:100DA0003197F1F744BB40E050E020E007C0A89540
:100DB0004F5F5F4F19F42F5F283019F083B38923F9
:100DC000B1F738BB37BB812F4AD9DC0121E030E0D5
:100DD000F9010090B30002C0EE0FFF1F0A94E2F782
:100DE00040917A0050E0B901042E02C0660F771FCF
:100DF0000A94E2F70090990002C0220F331F0A9470
:100E0000E2F78E2F862B822B84BB15BA440F551F19
:100E100082E090E002C0880F991F4A95E2F787BBF5
:100E200088BB362F6093800084EC99E00197F1F73E
:100E30002E2B24BBC0E0D0E0DD2408C0A89521966D
:100E400029F4D39428E0D21609F470C083B3832325
:100E5000A9F36CC0823009F070C065BB18BACD012F
:100E600002C0880F991FEA95E2F7982F80938000BF
:100E7000E4ECF9E03197F1F744BB45BB40E050E0CA
:100E800020E007C0A8954F5F5F4F19F42F5F28300F
:100E900019F083B38923B1F337BB812FE0D8DC018C
:100EA00021E030E0F9010090B30002C0EE0FFF1F17
:100EB0000A94E2F740917A0050E0B901042E02C092
:100EC000660F771F0A94E2F70090990002C0220F84
:100ED000331F0A94E2F78E2F862B822B84BB85BBAF
:100EE000440F551F82E090E002C0880F991F4A9579
:100EF000E2F787BB18BA362F6093800084EC99E044
:100F00000197F1F72E2B20938E0024BB25BBC0E068
:100F1000D0E0DD2407C0A895219621F4D39488E081
:100F2000D816A1F083B38323B1F710C0E3E8EE2E07
:100F3000E1E0FE2E012D112D0EC0C0E0D0E0A0E0BA
:100F4000B0E0EE24FF248701DD2405C07EE8E72E13
:100F5000F12C012D112D17BA18BA14BA15BA209711
:100F600011F4DD20F1F180917D00823031F48FEFBA
:100F700093E09C012A1B3B0BD90187E290E09C0186
:100F8000A29FC001A39F900DB29F900D112463E01A
:100F9000969587956A95E1F766E870E04AE050E03B
:100FA00080D56D2D70E080E090E0CB01772766273B
:100FB0009E0140E050E0620F731F841F951FA8013F
:100FC000970193D524E630E040E050E0C1D5C90157
:100FD0002330310508F003976FE870E04AE050E0F5
:100FE00060D5DF91CF911F910F91FF90EF90DF902F
:100FF0000895CF92DF92EF92FF920F931F93CF93BA
:10100000DF9380E481BB80EC82BB83E886B9ADD4FA
:1010100004B603FE0DC08CEE90E0F0D480E395E7BB
:1010200029E130E0F9013197F1F70197D9F74BC089
:1010300080E488D485EF90E0E1D480E883D4C6E8EA
:10104000D0E07FE8C72E70E0D72E04C09093B000A8
:101050008093AF008FE028E130E00FB6F894A895B8
:1010600021BD0FBE81BD10927E001092CC00109267
:101070007C0010927B0010927D001092AE001092C6
:101080007F006CD485E8EBD785E8E9D79093B00072
:101090008093AF008A58924038F58EE090E0AED44D
:1010A0008091AF009091B00088559240C0F480E2EA
:1010B00090E0A4D480E197E229E130E0F901319792
:1010C000F1F70197D9F712BA80E090E0DF91CF9164
:1010D0001F910F91FF90EF90DF90CF90089588E1DE
:1010E00090E08CD480EC2ED480E090E087D480E037
:1010F00061E042E09AD980E062E041E096D981E087
:1011000060E042E092D981E062E040E08ED982E086
:1011100061E040E08AD982E060E041E086D98091D8
:101120007E00882321F0863011F08130D1F418BA86
:1011300085E187BB84ED90E30197F1F717BA82E070
:1011400060E0C9D782E061E0C6D781E062E0C3D742
:1011500081E060E0C0D780E062E0BDD780E061E080
:10116000BAD7C8DDFBD380917E00813009F0C5C0BD
:1011700080917C00813019F581E590E03FD486EEC6
:1011800090E03CD48091B4008F5CDFD383E690E0A4
:1011900029D48091B5008F5CD8D380ECD3D38BED6C
:1011A00090E02CD48091B6009091B70066E870E092
:1011B0004AE050E034D416D483EE90E062C382302B
:1011C00009F052C03091B4002091B8003217E1F418
:1011D00089E590E013D487E690E004D480ECB2D3A4
:1011E00086EE90E00BD48091B4008F5CAED383EB9D
:1011F00090E004D48091B5008F5CA7D388EB90E099
:10120000FDD38091B90005C28091B5009091B900DD
:101210008917E1F489E590E0F1D38AE690E0E2D322
:1012200080EC90D38DE690E0DDD38091B5008F5CAB
:101230008CD389EA90E0E2D38091B4008F5C85D3AF
:101240008EEA90E0DBD38091B800E3C1821709F009
:101250000AC3931709F007C386E690E0CFD380EC6A
:1012600071D38FE690E00DC3833009F0FCC2809308
:101270007A00809399009091B4008091B8009817FB
:1012800021F08091BC00981711F490937A0090910E
:10129000B8008091BC00981711F490937A00909157
:1012A000B5008091B900981721F08091BD00981782
:1012B00011F4909399009091B9008091BD00981716
:1012C00011F49093990080917A00833008F0CBC29A
:1012D00080919900833008F0C6C286E690E08ED3F4
:1012E00080EC30D38CE790E089D380917A008F5CDA
:1012F0002CD383E690E076D38AC1823009F0F0C027
:1013000080917B00882381F48091AF009091B000A0
:101310009093B2008093B1008091A2009091A300BD
:101320009093A5008093A4002091AF003091B0006D
:101330008091B1009091B20082179307A0F430938E
:10134000B2002093B1008091A2009091A3009093ED
:10135000A5008093A400909199008091B3008093A0
:1013600099009093B30080917D00813019F482EC54
:1013700090E002C086EC90E041D38AEC90E03ED34E
:1013800080917A008F5CE1D28EEC90E037D380912F
:1013900099008F5CDAD282ED90E030D38091B30077
:1013A0008F5CD3D280ECCED26091B1007091B2004C
:1013B00080E090E023EB32E040E050E096D3609391
:1013C000A6007093A7008093A8009093A900809135
:1013D000A4009091A5000B9730F48BE090E09093DF
:1013E000A5008093A4002091A4003091A50040E0C6
:1013F00050E06091A6007091A7008091A8009091A4
:10140000A900A6D32093A6003093A7004093A8007C
:101410005093A900C9012093B1009093B2008DEBC5
:1014200090E0ECD28091B1009091B20066E870E05B
:101430004AE050E036D3D6D287EC84D280917C004B
:10144000833010F080E001C080E27FD210929900DA
:101450003FC0A22FB0E0FD01EE0FFF1FEE0FFF1FF8
:10146000EC54FF4F41813091B300431749F4908110
:1014700080917A00981721F480917D00813089F065
:10148000AA0FBB1FAA0FBB1FAC54BF4F8C91831771
:10149000E1F480917A004817C1F480917D00823098
:1014A000A1F48BED90E0AAD2E0919900F0E0EE0F6C
:1014B000FF1FEE0FFF1FEC54FF4F8281938166E800
:1014C00070E04AE050E0ABD272C02F5F20939900E9
:1014D0002091990080917C00281708F4BACFE4C1CC
:1014E000833009F067C080917D0080FF02C08EE4E8
:1014F00001C080E52AD290917D00892F83508230EF
:1015000018F480E990E008C09550923018F483E90F
:1015100090E005C08DE890E071D288E890E06ED24E
:1015200080917D008330E0F48BE191E067D2F60199
:1015300001900020E9F73197EF58F040E0938000E8
:10154000E0938E00E53018F084E0809380008FE80F
:1015500090E06091800040918E0090DB8EE6F5D1A6
:1015600080ECF0D186ED90E049D280917A008F5CDA
:10157000ECD1809199008F5CE8D18091B3008F5CB1
:10158000E4D180917C00882331F080917D0083300C
:1015900010F480E001C080E2D8D180917D008330DA
:1015A00008F082C18FED90E029D286E890E01AD24F
:1015B0008DE679C1853099F489E990E01FD280ECFD
:1015C000C1D180E790E00ED280917A008F5CBDD1CE
:1015D000809199008F5CB9D18091B3001AC084309A
:1015E000D1F483EA90E00AD280ECACD189EE90E0AD
:1015F00005D280917A008F5CA8D189EA90E0FED173
:101600008091B3008F5CA1D18EEA90E0F7D18091F8
:1016100099008F5C48C1863009F0D0C08BE091E022
:10162000EDD18091CD008F5C90D18DE28ED18091F3
:1016300085008F5C8AD180EC85D185E790E0D2D19E
:101640002091AA003091AB0082E02130380738F0B9
:10165000205032403093B0002093AF0008C080E0AB
:1016600092E0821B930B9093B0008093AF00209187
:10167000AC003091AD0082E02130380738F02050C6
:1016800032403093B2002093B10008C080E092E075
:10169000821B930B9093B2008093B1002091AF0016
:1016A0003091B0008091B1009091B2008217930701
:1016B00098F4809197009091980090939600809371
:1016C00095008091AC009091AD009093AB00809319
:1016D000AA008CE592E102C088EA92E09093AD0006
:1016E0008093AC008091AA009091AB00892B31F4DB
:1016F00081E090E09093AB008093AA00E090AA0074
:10170000F090AB0000E010E02091AC003091AD0013
:1017100040E050E0C801B701E8D120919500309138
:10172000960040E050E02E193F09400B510B10D2BB
:10173000CA012093A6003093A7004093A80090937D
:10174000A900B90146E850E02AE030E087D1809155
:10175000AC009091AD008C55924159F5FE0101907D
:101760000020E9F73197E658F040E093CD00109261
:10177000850016C0F0E0EA57FF4F8081E6D0209147
:10178000850030E08091CD0090E00297281739075E
:1017900011F48EE2DAD0809185008F5F809385000E
:1017A000E09185008091CD00E81720F38BE6CDD045
:1017B00003C086E890E016D184EF75C0873009F049
:1017C00052C08FE191E01AD18091AE008F5CBDD004
:1017D0008DE2BBD080917F008F5CB7D080ECB2D01F
:1017E0008EE680938E0060918100709182008091DE
:1017F000830090918400603A26E8720721E0820716
:1018000020E0920780F028EE33E040E050E0A0D1E5
:101810002093810030938200409383005093840092
:1018200084EE80938E00609181007091820080919F
:1018300083009091840046E850E02AE030E00ED129
:10184000FE0101900020E9F73197E658F040E0935F
:10185000800086E890E06E2F4E2F10DA80918E0087
:1018600074D086E420C080917C00882361F486E2F5
:1018700090E0C4D080EC66D087E390E0BFD081E4F4
:1018800090E0BCD011C081E490E0B8D089E490E051
:10189000B5D080EC57D08EEF90E0B0D080917C0036
:1018A000805D53D080E051D0879BFECF80E593ECE4
:1018B0000197F1F71092B0001092AF0080E090E035
:1018C0004AEF50E00AC09C012F5F3F4F879BBECB81
:1018D000A895CA010197F1F7C90127E28031920763
:1018E00090F39093B0008093AF00969888E10FB684
:1018F000F89481BD11BC0FBE8799FECFABCB92B3DC
:10190000282F22952F70907F292B22BB31E0932F17
:101910009A95F1F7959A23E0922F9A95F1F7959879
:1019200092B38F70907F982B92BB3A95F1F7959A6E
:101930002A95F1F7959884E18A95F1F782B3807F33
:1019400082BB08959498DBDF0895949AD8DF0895B8
:10195000959A83E08A95F1F79598089581E0F2DFF2
:1019600082EE94E00197F1F7089581B38F6381BB14
:101970008CE49DE10197F1F782B3807E836082BBA6
:10198000959A93E0892F8A95F1F79598E2EEF4E025
:101990003197F1F7959A892F8A95F1F795982AEF63
:1019A00030E0F9013197F1F7959A892F8A95F1F78F
:1019B0009598F9013197F1F782B3807E826082BBFE
:1019C000F9013197F1F7959A9A95F1F79598C90130
:1019D0000197F1F788E2B6DF8CE0B4DF86E0B2DF92
:1019E000BDDF0895CF93DF93EC0102C0AEDF2196F7
:1019F00088818823D9F7DF91CF910895CF93DF9322
:101A0000EC01E199FECFDFBBCEBBE09A8DB388231A
:101A100019F09BDF2196F5CFDF91CF910895FB015F
:101A20009F01E8944230BCF04532ACF44A3029F4CE
:101A300097FB1EF4909581959F4F642F772774D064
:101A4000805D8A330CF0895D8193CB010097A9F703
:101A500016F45DE251931082C90137C0FA01CF93A9
:101A6000FF93EF932230C4F02532B4F4C22F2C2F11
:101A7000332744275527FF93EF936AD0EF91FF91C7
:101A8000605D6A330CF0695D6193B901CA01605011
:101A900070408040904059F710828F919F91CF9174
:101AA00014C0FB019F0142306CF045325CF4642F9E
:101AB00077273AD0805D8A330CF0895D8193CB0122
:101AC0000097A9F71082C90100C0DC01FC01672F53
:101AD00071917723E1F7329704C07C916D93708305
:101AE0006291AE17BF07C8F30895629FD001739F3C
:101AF000F001829FE00DF11D649FE00DF11D929FAA
:101B0000F00D839FF00D749FF00D659FF00D9927E8
:101B1000729FB00DE11DF91F639FB00DE11DF91F0C
:101B2000BD01CF0111240895AA1BBB1B51E107C0C1
:101B3000AA1FBB1FA617B70710F0A61BB70B881F5D
:101B4000991F5A95A9F780959095BC01CD010895EC
:101B5000A1E21A2EAA1BBB1BFD010DC0AA1FBB1FB1
:101B6000EE1FFF1FA217B307E407F50720F0A21B23
:101B7000B30BE40BF50B661F771F881F991F1A9490
:101B800069F760957095809590959B01AC01BD01BA
:081B9000CF010895F894FFCF86
:101B9800302E003B4B3D004341004343004B3D008A
:0A1BA80047414B3D0052203D200054
:00000001FF
